:100000000C942A000C9445000C9445000C94450077
:100010000C9445000C9445000C9445000C9445004C
:100020000C9445000C9445000C9445000C9447003A
:100030000C9445000C9445000C9445000C9445002C
:100040000C9445000C9445000C9445000C9445001C
:100050000C94450011241FBECFE5D4E0DEBFCDBF18
:1000600011E0A0E6B0E0E0E9F7E002C005900D92F3
:10007000A43EB107D9F712E0A4EEB1E001C01D9291
:10008000AC3BB107E1F70C9469030C9400001F929C
:100090000F920FB60F9211242F938F939F93EF938C
:1000A000FF935C9B02C084E00BC02CB190913302A3
:1000B0009657923010F0109276025B9B04C083E05A
:1000C000809332021BC0809131028B3418F083E69A
:1000D0008093320280913102E82FFF27EC51FE4FCE
:1000E0002083809131028F5F80933102923030F40F
:1000F00080913102813410F010927602FF91EF91DD
:100100009F918F912F910F900FBE0F901F90189578
:1001100088E98AB983E389B910922F0210923002DC
:100120001092310208955D9BFECF8CB908950000B6
:1001300000000000000000000000000000000000BF
:10014000000000000000019791F7089500000000F2
:1001500008958FB9779BFECF08951F93CF9384E1C5
:100160008DB990E898BB8FE987BB10E098BBC79822
:10017000C79AC12FC7980E94A600C79AB599116067
:10018000C73008F4110FCF5FC830A0F3C798C79AE3
:10019000C79880E888BBC7988FEB87BB84E58DB98B
:1001A000812F9927CF911F910895982F85E08FB9BE
:1001B000779BFECF905E9FB9779BFECF0E94AD00EC
:1001C000992708950F931F93182F062F84E00E94FC
:1001D000A900812F0E94A900802F0E94A90080E021
:1001E0000E94A9001F910F910895AC0120E02617ED
:1001F00050F4FA01E20FF11D80818FB9779BFECF99
:100200002F5F2617B0F3089584E18DB918BA8FE1F6
:1002100087BB81E08CBF89E183BFB59BFECFB599D9
:10022000FECF8AE090E00E94970013BE18BA8FEBD1
:1002300087BB84E58DB9089563E084E291E00E9474
:10024000F50064E288E291E00E94F5000E9404015A
:1002500008950F931F93CF93C0E005E312E0C05EB3
:10026000F80161918F018C2F0E94E200CF51C034C0
:10027000B0F3CF911F910F9108950F931F93CF93D8
:10028000C0E005E312E08C2F8058F80161918F01E6
:100290000E94E200CF5FC034B0F3CF911F910F9165
:1002A00008950F931F938C0163E084E291E00E9414
:1002B000F500602F8AEF0E94E20064E28DE491E095
:1002C0000E94F5000E9404011F910F910895682F6C
:1002D0008AEF0E94E20064E282E791E00E94F5006A
:1002E0000E940401089563E084E291E00E94F50019
:1002F00064E287E991E00E94F5000E9404010895FC
:100300000F931F9367E28CEB91E00E94F5000E942F
:10031000040162E08FE191E00E94F5000E94AD00CF
:100320009927182F002762E081E291E00E94F500F2
:100330000E94AD009927082B192BC8011F910F911E
:100340000895A89A8EE190E00E949700A8988EE107
:1003500090E00E94970060E380E690E00E94F50044
:100360000E94040167E281E990E00E94F5000E948A
:10037000040169E389EB90E00E94F50067E283EFF6
:1003800090E00E94F5000E94040162E08BE191E0A0
:100390000E94F5000E94AD008093BB0262E08DE1F7
:1003A00091E00E94F5000E94AD00809379020895CB
:1003B0000F931F93CF93DF938091BB028823F1F4B7
:1003C000809179028530D0F400E010E088EE93E06F
:1003D0000E949700C8010E946701C0E0D0E08C2F06
:1003E0000E94D5000E9493002196C034D105BCF331
:1003F0000F5F1F4F0F3F110549F344F381E08093D6
:1004000076028FE680933302DF91CF911F910F9197
:100410000895AF92BF92CF92DF92EF92FF920F9327
:100420001F93CF93DF938FE60E94930081E0809328
:100430007602809176028130E1F38091E401A82E6A
:10044000BB2481E080937602109231021092340234
:100450008091BB02882309F082C0809179028530A7
:1004600008F07DC00E941C0100E010E08FE60E94B1
:10047000930081E080937602809131028034E0F332
:10048000E5E3F2E0A4EEB1E09F01215C3F4F8D91E6
:1004900081932E173F07DCF70E942901C8010E94B3
:1004A0005101C8010E946701C0E0D0E045E3C42EBD
:1004B00042E0D42E3AE7E32E32E0F32E8C2F0E9456
:1004C000D500982FF70181937F01F60181916F018B
:1004D000891719F081E0809334022196C034D10548
:1004E0006CF3109231020E94A6000F5F1F4FA016FE
:1004F000B1060CF0BBCF80913402882311F48FE653
:1005000001C088E70E9493008FE6809333028091B8
:100510007702909178024097B1F480917602813011
:10052000E1F710927602E5E3F2E0A4EEB1E09F017C
:10053000215C3F4F8D9181932E173F07DCF70E947E
:100540003D010E947301809177029091780280971B
:1005500031F4809176028130E1F710927602DF91DA
:10056000CF911F910F91FF90EF90DF90CF90BF90B0
:10057000AF900895AF92BF92CF92DF92EF92FF9229
:100580000F931F93CF93DF938FE60E94930081E038
:1005900080937602809176028130E1F38091E401CC
:1005A000A82EBB2481E08093760210923102109233
:1005B00034028091BB02882309F052C080917902F5
:1005C000853008F04DC000E010E08FE60E949300F7
:1005D00081E080937602809131028034E0F3E5E39C
:1005E000F2E0A4EEB1E09F01215C3F4F8D91819339
:1005F0002E173F07DCF7C8010E946701C0E0D0E07A
:1006000065E3C62E62E0D62E5AE7E52E52E0F52EBF
:100610008C2F0E94D500982FF70181937F01F6015E
:1006200081916F01891719F081E08093340221963E
:10063000C034D1056CF3109231020E94A6000F5F06
:100640001F4FA016B1060CF680913402882311F4D6
:100650008FE601C088E70E9493008FE68093330203
:10066000DF91CF911F910F91FF90EF90DF90CF908E
:10067000BF90AF9008950E9480010E94930080ED8A
:1006800097E00E94970080E00E9493000895A89A46
:100690008EE190E00E949700A8988EE190E00E9481
:1006A000970008959FEF9ABB8FEB87BB94BB91BBDC
:1006B0001BBA18BA15BA12BA84E58DB9A89A9093E4
:1006C000BB02909379021092340281E0809376020B
:1006D0000895CFE5D4E0DEBFCDBF0E9452030E9453
:1006E0008800789490917602992309F04FC0809108
:1006F000E401809333029093310299278F3691055C
:10070000E1F1803791058CF48536910551F18636FB
:10071000910524F48336910569F131C0893691053C
:10072000C9F08E36910591F02AC08337910551F1B9
:100730008437910524F48237910581F020C08637F3
:100740009105A9F08737910579F019C00E94A101A0
:100750008EE616C080917902805D12C00E94D80199
:1007600011C00E941C0109C00E9409020BC00E9416
:10077000BA0208C00E943B0305C08FE601C088E7AB
:100780000E94930081E080937602A99AA998AACF4B
:1007900032800000000000000023D90037B8003785
:1007A000B04027C1D027C85837A80037A01827D98C
:1007B0000037C98037D20037804037C0001BFC4863
:1007C0003037B80037B04027C1D027C85837A80005
:1007D00037A01827D90037C98037D20027D008376B
:1007E000803037C00037F8902737B80037A0183767
:1007F000A80037B04037C28837CFE037D18037FF05
:100800009000000037B80037A01837A80037B04074
:1008100037C30037CF5037D18037B88037F89000D2
:1008200000003937B80037B04027C1D027C8583743
:10083000A80037A01827D90037C98037D20027D0A1
:100840000037803037C00037F8902705F805F917D2
:10085000E417E00227E0680337B80037B20027C189
:10086000D027CA1837A80037A01827DC0037C9805E
:1008700037D20037802837C00037F8902437B800C7
:1008800037B04027C1D027C85837A80037A018274D
:10089000D90037C98037D20037801037C00037F809
:1008A000902437B80037B04027C1D027C85837A8A0
:1008B0000037A01827D90037C98037D20037800801
:1008C00037C00037F8902437B80037B20027C1D0BE
:1008D00027CA1837A80037A01827DC0037C9803787
:1008E000D20037802037C00037F8902437B800375F
:1008F000B04027C1D027C85837A80037A01827D93B
:100900000037C98037D20027D00037803837C00081
:0409100037F89027FD
:00000001FF
